:100000000C9496020C94CE020C94CE020C94CE0268
:100010000C94CE020C94CE020C94CE020C94CE0220
:100020000C94CE020C94CE020C94A6220C94752350
:100030000C94861D0C94CE020C94CE020C94CE022D
:100040000C94CE020C94CE020C94CE020C94CE02F0
:100050000C94CE020C940E1E0C94CE020C94CE0284
:100060000C94CE020C94CE020C94CE020C94CE02D0
:100070000C94CE020C94CE020C94CE020C94CE02C0
:100080000C94CE020C94CE020C94CE020C94CE02B0
:100090000C94CE020C94CE020C94CE020C94CE02A0
:1000A0000C94CE020C94CE020C94CE0201080108EE
:1000B0002D082D089508B308CB09CB09BE085709B0
:1000C000680968098D1A831A901AD81ADC1ADC1A82
:1000D000D81ADC1ADC1AB11ADC1ABB1AC51ADC1AD7
:1000E000DC1ADC1ADC1AD81ADC1ADC1AD81ADC1A68
:1000F0009E1ADC1ADC1AD51AD51AD51AD51AD51AB1
:10010000D51AD51AD51AD51ADA1ADC1A8D1A801A08
:10011000DC1ADC1ADC1ADC1ADC1ADC1ADC1ADC1A2F
:10012000DC1ADC1ADA1ADC1ADC1AD81ADC1AD31A2E
:10013000D31AD31AD31AD31AD31AD31AD31AD31A57
:10014000DA1AE223092401250924012555247824FB
:100150000125CF24DE240102E0630103E001014F09
:100160000102E0760103E0004B6579626F61726421
:1001700000437573746F6D005468650029000000BA
:100180003A003B003C003D003E003F004000410083
:100190004200430044004500460047004800350047
:1001A0001E001F0020002100220023002400250043
:1001B000260027002D002E002A0049004A004B008F
:1001C0002B0014001A000800150017001C0018006E
:1001D0000C00120013002F00300031004C004D00C5
:1001E0004E00390004001600070009000A000B0049
:1001F0000D000E000F003300340000002800000046
:1002000000000000E1001D001B00060019000500B1
:100210001100100036003700380000000000E50033
:10022000000052000000E000E300E20000000000D7
:100230002C0000000000E6000000E7000000015173
:10024000E400500051004F00C15C0000A75DA85DB4
:10025000A95DA95DAA5DAB5DAC5DAD5DAE5DAF5D59
:10026000B05DB15D0100010001000100010001006D
:100270000100010001000100010001000100010076
:100280000100010001000100010001000100010066
:100290000100010001000100010001000100010056
:1002A0000100010001000100010001000100010046
:1002B0000100010001000100010001000100010036
:1002C000010001000100000001000000000000002A
:1002D0000100010001000100010001000100010016
:1002E0000100010001000000000001000000010009
:1002F00000000100010001000000000001000000FA
:1003000000000100000001000000010001000100E8
:100310000100010000000000000000002A2B28005E
:1003200000000000000000000000000000000029A4
:10033000000000002C1E3420212224342627252EE4
:10034000362D3738271E1F2021222324252633331C
:10035000362E37381F0405060708090A0B0C0D0E48
:100360000F101112131415161718191A1B1C1D2F14
:100370003130232D350405060708090A0B0C0D0E34
:100380000F101112131415161718191A1B1C1D2FF4
:100390003130354C0000000000000000000000007B
:1003A000000000000000000000000000000000004D
:1003B00000000000000000007E0F00D4FFFFFFC718
:1003C000000000780A034B004D004100430000008C
:1003D00012034B00420044004D0061006E006900B2
:1003E000610000000403090409023B00020100A0AF
:1003F000FA090400000103010100092111010001B3
:1004000022400007058103080001090401000103DF
:1004100000000009211101000122B6000705820336
:1004200020000112010002000000084D4B4341046E
:10043000010102000105010902A10185020901A1D2
:100440000005091901290815002501950875018184
:10045000020501093009311581257F950275088152
:100460000609381581257F950175088106050C0A56
:1004700038021581257F950175088106C0C00501E8
:100480000980A101850319012AB700150126B700CB
:10049000950175108100C0050C0901A101850419A1
:1004A000012AA002150126A002950175108100C045
:1004B00005010906A1018506050719E029E71500D0
:1004C00025019508750181020507190029EF15001E
:1004D000250195F075018102050819012905950589
:1004E00075019102950175039101C005010906A1ED
:1004F00001050719E029E715002501950875018117
:10050000029501750881010507190029FF150026CC
:10051000FF00950675088100050819012905950554
:1005200075019102950175039101C00011241FBE50
:10053000CFEFDAE0DEBFCDBF04B603FE18C0809176
:10054000050390910603A0910703B091080387303B
:10055000904BA740B04B59F410920503109206033C
:100560001092070310920803E0E0F8E3099511E008
:10057000A0E0B1E0E8E6FBE402C005900D92A239EC
:10058000B107D9F723E0A2E9B1E001C01D92A5307F
:10059000B207E1F70E94E0140C94B2250C9400001D
:1005A000CF93DF93A9E1B1E04FE151E061E070E06A
:1005B0008D91E82FE295EF70F0E021A18F70EB01B3
:1005C00002C0CC0FDD1F8A95E2F7CE01922F982B47
:1005D00091A392A18095892382A34A175B0741F7D3
:1005E000DF91CF91089508950C94F3020C94F402D6
:1005F0000C94F30224E0829FC0011124FC01EC560C
:10060000FE4F6081718182819381089508950E94D7
:10061000D002AAE2B1E041E050E08D91E82FE295EE
:10062000EF70F0E021A18F70BA0102C0660F771F52
:100630008A95E2F7CB01962F9095922391A392A1F0
:10064000892B82A371E0A033B70739F76A98729AB1
:10065000ECEAF1E0A4E9B1E0119211921192119249
:100660001D921D921D921D9281E0E43CF807A1F7B6
:1006700086E00E9497140C94A9042F923F924F9207
:100680005F926F927F928F929F92AF92BF92CF9222
:10069000DF92EF92FF920F931F93CF93DF9300D0DF
:1006A00000D01F92CDB7DEB71B821A8210E04A81BC
:1006B00049834031E1F0842F885F84FF02C02E9A85
:1006C00001C02E9883FF02C0469A01C0469882FF5F
:1006D00002C0479A01C0479881FF02C0899A01C0B1
:1006E000899880FF02C0889A03C0889801C02D9A1B
:1006F00050E55A95F1F7C12CD12C7601C3940A80AC
:1007000004C0CC0CDD1CEE1CFF1C0A94D2F7460181
:10071000570180949094A094B0948CEA91E09D83CA
:100720008C832AE231E000E060E06C807D80F301A0
:1007300080819181A281B381633071F4F981F111DB
:100740000BC01C012D01629904C0689420F8F301CC
:1007500021C0E89420F81CC0F9017081472F429510
:100760004F7050E0FA0140A150E07F7002C05595F3
:1007700047957A95E2F71C012D0140FD05C0282020
:1007800039204A205B2004C02C283D284E285F28B1
:10079000EC81FD8120823182428253824C815D81D5
:1007A0004C5F5F4F5D834C83F3012080318042803A
:1007B000538082159305A405B50509F001E06F5F2C
:1007C0002F5F3F4F663009F0B0CF0E94D002102B50
:1007D0004A815B814F5F5F4F5B834A8341315105A3
:1007E00009F065CF212F46E064E971E08CEA91E0E1
:1007F0000E9498140E94AB04812F0F900F900F90CD
:100800000F900F90DF91CF911F910F91FF90EF907C
:10081000DF90CF90BF90AF909F908F907F906F9020
:100820005F904F903F902F900895219A229A239A9B
:10083000249A579A089580FF02C0299A01C02998E6
:1008400081FF05C02A982B982C985F9808952A9AC2
:100850002B9A2C9A5F9A0895FB01883A2DE592070E
:1008600099F020F4873A9D4549F021C0893A2DE559
:10087000920781F08A3A9D4599F019C082818823B8
:10088000B1F088E791E011C08281882381F081E78F
:1008900091E00BC08281882351F088E691E005C089
:1008A0008281882321F086E591E00E94F60581E0AF
:1008B000089581E008950C942C0408950C945D042F
:1008C0001F93CF93DF9300D000D01F92CDB7DEB738
:1008D00049835A836B833091C50189819A81311193
:1008E00014C0662359F0222349F00E94080C182FE7
:1008F000682F89819A810E94B10B03C00E94DC0B92
:10090000182F69817A81812F04C00E94080C6981A7
:100910007A810F900F900F900F900F90DF91CF91F1
:100920001F910C946A13FC01262F40815181628132
:10093000738184810C94600481E00895CF93DF93E8
:10094000EC0160E00E949304BE01DF91CF910C9412
:100950005E040C94F6020C94F80208950E945B0A5F
:100960000E94AD042FE78AE196E02150804090403C
:10097000E1F700C000000C94341E0F931F93CF9337
:10098000DF938C0161E00E949304EC01B8010E94A6
:100990005B04882309F444C0B801CE010E946318A7
:1009A0008823F1F1B801CE010E94CF1B8823C1F149
:1009B000B801CE010E949318882391F1B801CE01AD
:1009C0000E942B1B882361F1F8018281882309F1A1
:1009D000CB358DE5D807C1F050F4C115FCE5DF0734
:1009E00081F0CF3DDC45A9F40E943F1119C0CC3500
:1009F000EDE5DE0761F0CD35DD4559F40E9482104A
:100A000008C00E94AE040CC00E948B1002C00E945D
:100A10008E10C801DF91CF911F910F910C94590452
:100A200080E0DF91CF911F910F9108950E94661D84
:100A300080E00E941B040C941F060E9487170E94EE
:100A400022060C946C1DDF92EF92FF920F931F937E
:100A5000CF93DF93E82FF0E0EC5EFC4FD490282F8B
:100A600026952695269530E0F901EC54FC4F04912B
:100A7000877010E0082E02C0159507950A94E2F7DA
:100A800001701127F901EC55FC4FE490F12C082E70
:100A900002C0F594E7940A94E2F791E0E922FF247A
:100AA000F901EC56FC4FC491D0E002C0D595C79532
:100AB0008A95E2F7C170DD270115110519F081EE65
:100AC0000E948106E114F10419F086EE0E9481066D
:100AD0008D2D0E94AF07EF2819F086EE0E94300797
:100AE000012B19F081EE0E943007CD2B51F08CE2E2
:100AF000DF91CF911F910F91FF90EF90DF900C94B9
:100B0000AF07DF91CF911F910F91FF90EF90DF9092
:100B10000895EF92FF920F931F93CF93DF938C0171
:100B2000F62E8AE0E82EF8018491882309F457C054
:100B3000813009F042C0E8012196FE0184918130A4
:100B400031F42196FE0184910E94AF0739C08230B2
:100B500039F4E8012296FE0184910E94810630C09A
:100B6000833039F4E8012296FE0184910E94300717
:100B700027C0843029F5E8012296FE01249180E007
:100B800090E030E0205331092A30310560F4E89ECE
:100B9000A001E99E500D1124C901840F951F2196D3
:100BA000FE012491EECF009759F0EFECF7E031977A
:100BB000F1F700C000000197F6CF0E942305E8017D
:100BC0008E010F5F1F4F8F2D882309F4ACCFEFEC00
:100BD000F7E03197F1F700C000008150F5CFDF91C9
:100BE000CF911F910F91FF90EF90089560E00C94CA
:100BF000890508950C94F90581E00895CF93C82FD5
:100C00000E94FC05882359F0C095C1FF02C0289AB4
:100C100001C02898C2FF02C0769A01C07698CF9191
:100C20000895209A289A6E9A769A0895CF93C82F9D
:100C30000E94FA058C2F0E94FE05CF91089580E056
:100C40000C9416060E942B1C0C9416060E942B1C5A
:100C50009091C401891721F08093C4010C94160669
:100C60000895CF93DF93CDB7DEB72B970FB6F894E7
:100C7000DEBF0FBECDBF4F83588769877A878B87CA
:100C800061110E94CE0F9E012F5F3F4F86E0F90158
:100C900011928A95E9F785E0FE013796D901019016
:100CA0000D928A95E1F789819A814C815D81452B6E
:100CB00031F09F3F31F491E08F3F19F403C091E090
:100CC00001C090E090FF09C049815A816B817C810D
:100CD0008D819E810E94EF0E05C0C9010E949C0477
:100CE0008111F2CF2B960FB6F894DEBF0FBECDBFA9
:100CF000DF91CF910895FC01808191810E944A0C7F
:100D00000895CF93882309F4A9C0C82F8238C1F46D
:100D10000E942B1C81FDA2C069E380910201909189
:100D200003010E94211D0E94F00F2FEF80E792E047
:100D3000215080409040E1F700C0000069E319C0F5
:100D4000833801F50E942B1C80FD88C063E58091EB
:100D50000201909103010E94211D0E94F00F2FEFCC
:100D600080E792E0215080409040E1F700C0000011
:100D700063E580910201909103010E942C1DCF91A7
:100D80000C94F00F8438C1F40E942B1C82FD66C0C5
:100D900067E480910201909103010E94211D0E944D
:100DA000F00F2FEF80E792E0215080409040E1F774
:100DB00000C0000067E4DDCF8CEF8C0F813AF8F4BF
:100DC0008C2F0E94E21A811149C06C2F8091020180
:100DD000909103010E94A11C882349F06C2F8091FF
:100DE0000201909103010E942C1D0E94F00F6C2FB4
:100DF00080910201909103010E94211DC0CF80E2E9
:100E00008C0F883048F4C77081E001C0880FCA9504
:100E1000EAF70E94B10FB3CFEBE5EC0FE33040F4FB
:100E2000F0E0E25AFE4F808190E0CF910C945F1C7D
:100E3000E8E5EC0FE73150F4F0E0EE0FFF1FE05D66
:100E4000FE4F80819181CF910C94751CCD3E30F086
:100E50008C2F0E946515CF910C943716CF91089571
:100E6000882309F464C0823879F40E942B1C81FF26
:100E70005EC069E380910201909103010E94211DEF
:100E80000E94F00F69E310C08338B1F40E942B1C5C
:100E900080FF4DC063E580910201909103010E94A3
:100EA000211D0E94F00F63E58091020190910301E2
:100EB0000E942C1D0C94F00F843879F40E942B1C96
:100EC00082FF35C067E480910201909103010E9486
:100ED000211D0E94F00F67E4E7CF9CEF980F913A35
:100EE00010F4682FE1CF90E2980F983050F487709B
:100EF00091E001C0990F8A95EAF7892F0E94B70FF8
:100F0000D9CF9BE5980F933020F480E090E00C94CB
:100F10005F1C98E5980F973120F480E090E00C94E6
:100F2000751C8D3E20F00E94C0150C943716089554
:100F30001F93CF93DF93182FEB010E948106209718
:100F400041F08FEC97E00197F1F700C00000219786
:100F5000F6CF812FDF91CF911F910C943007893309
:100F600019F060E070E002C060E570E00C94980752
:100F7000882321F00E94B10F0C94F00F089588236C
:100F800021F00E94B70F0C94F00F0895CF92DF92DA
:100F9000EF92FF920F931F93CF93DF937C01D62F95
:100FA000C72FFC011281058102950F700E94A70FC7
:100FB0008823B9F01123A9F08C2F807F803421F091
:100FC00080E28D0F883068F08091F20282FD09C0C6
:100FD00082E00E9450100E94A70F91E0D82ED926DF
:100FE00001C0D12CCC2EC2948FE0C8228C2D90E071
:100FF0008C30910508F0CFC1FC01EA5AFF4F0C94E8
:1010000049258C2F807FCF70882311F0C295C07F37
:10101000112399F0CC2309F4AAC180E28D0F883006
:1010200010F0D11104C08C2F0E94B10F03C08C2F7F
:101030000E94C10F0E94F00F9AC18D2F0E943007AD
:10104000CC2309F4A8C180E28D0F883038F1DD236C
:1010500029F18C2F0E94C70F24C08C2F807FCF7066
:10106000803211F0C295C07FDD2319F0D130A1F19B
:101070003DC08091F20282FF17C0112349F0CC23BA
:1010800029F08C2F0E94B10F0E94F00F80E070C1F8
:1010900080E00E943007CC2309F47DC18C2F0E9490
:1010A000B70F0E94F00F77C1112371F0002341F0B8
:1010B000013031F40E94D10F8C2B0E94D90F6BC1EB
:1010C0000E94D10F8C2B1DC0002319F0013009F4B0
:1010D00062C10E94E60F25C0112321F0063008F0FE
:1010E0005AC10EC0053008F056C11BC0112361F073
:1010F000002331F0F701858180FF39C18F7085832E
:101100008C2F0E94B80747C1002359F0D93309F04A
:101110003FC1FFEF03EF11E0F15000401040E1F755
:1011200035C18C2F0E94BF0736C18C2F86958695BE
:10113000837019F0813061F02EC1112321F08D2FC1
:101140009C2F937002C080E090E00E945F1C2BC136
:10115000112321F08D2F9C2F937002C080E090E02E
:101160000E94751C20C18D2F112319F00E94651556
:1011700002C00E94C0150E94371615C18C2F8370C3
:1011800009F047C011110BC12D2F2295269527700C
:10119000220F220F6D2F6F70862F90E0A0E0B0E03D
:1011A000022E04C0880F991FAA1FBB1F0A94D2F7F2
:1011B000D4FF10C04FE050E060E070E004C0440F86
:1011C000551F661F771F2A95D2F740955095609559
:1011D000709503C040E050E0BA01C695C695C37053
:1011E0008A019B01082B192B2A2B3B2BC901B80123
:1011F000C23049F058F4C13019F00E94C70ACFC07C
:101200000E94B50ACCC00E94D90AC9C00E94B30A84
:10121000C6C0112319F08C2F817001C086958823D8
:1012200009F4BDC02D2F229526952770220F220F7D
:101230006D2F6F70862F90E0A0E0B0E0022E04C00A
:10124000880F991FAA1FBB1F0A94D2F7D4FF10C0A2
:101250004FE050E060E070E004C0440F551F661F8F
:10126000771F2A95D2F7409550956095709503C0E9
:1012700040E050E0BA01C695C695C3708A019B0153
:10128000082B192B2A2B3B2BC901B801C23049F07E
:1012900058F4C13019F00E948C0B81C00E947A0B67
:1012A0007EC00E949E0B7BC00E94ED0A78C0CF706A
:1012B000112339F08C2F0E94130B8D2F0E94B80739
:1012C0006EC08D2F0E94BF078C2F0E94340B67C009
:1012D000D23F21F128F4D03F41F0D13FC1F043C0CB
:1012E000D33F19F1D43F79F03EC0112341F00530CE
:1012F00008F051C08C2F8F710E94590B4CC00630E2
:1013000008F049C0F7CF8091F20282FF18C0112384
:1013100039F08C2F8F710E94130B3DC01123C9F33C
:101320008C2F8F710E94340B36C0112329F08C2F23
:101330008F710E94FE0A2FC00E94F90A2CC011234F
:1013400049F0CF718C2F0E94130B63E08C2F0E9409
:10135000351021C081E00E9450100230E0F082E0A0
:101360000E94501018C0112331F0002391F28D2FEC
:101370000E94810610C0002399F2D93349F41FEF6F
:1013800023EF31E0115020403040E1F700C0000071
:101390008D2F0E94300788EF8C0D843020F40E943E
:1013A0002B1C0E941606DD20C9F00E94A30F80FDB1
:1013B00015C0F70112820E949D0F0E94130BC701F6
:1013C0000E940F0A0E949D0FDF91CF911F910F91F4
:1013D000FF90EF90DF90CF900C94340BDF91CF9182
:1013E0001F910F91FF90EF90DF90CF9008950F9392
:1013F0001F93CF93DF93EC01688179818A810E94EA
:10140000550C8C010E94B00B0E94A10AB801CE01BC
:101410000E94C607DF91CF911F910F910895CF933E
:10142000DF93EC01988189812B813C81232B31F062
:101430008F3F31F481E09F3F19F403C081E001C088
:1014400080E080FD1DC0CE010E94BD04811110C04E
:101450000E94A70F8823A1F08A81882389F08091B8
:10146000F20282FD0DC082E0DF91CF910C9450100A
:10147000CE010E94F709CE01DF91CF910C949E041A
:10148000DF91CF91089580E090E00E945F1C80E0A2
:1014900090E00E94751C0E94CE0F0E94F00F0E94E7
:1014A00068170C94371680910201909103010E94F5
:1014B000371D0C94430A0E94BE0F0C94530A929558
:1014C0009F70963079F010F4925001C09A5092308B
:1014D00068F4803F69F018F4883E40F409C0843F06
:1014E00029F406C0883E20F0813F11F080E0089585
:1014F00081E00895FC01808191810E944A0C0E9444
:101500005F0A0895CF93DF9300D000D01F92CDB72C
:10151000DEB70F900F900F900F900F90DF91CF914B
:101520000895CF93DF9300D000D000D0CDB7DEB7C1
:1015300026960FB6F894DEBF0FBECDBFDF91CF91D8
:101540000895089508950C94A20A0C94A30A0E9489
:10155000A50A60930B0270930C0280930D02909386
:101560000E020C94430A0C94A70A0F931F93009148
:101570000B0210910C0220910D0230910E02602B93
:10158000712B822B932B1F910F910C94A70A0F9311
:101590001F9300910B0210910C0220910D023091CB
:1015A0000E0260237123822393231F910F910C94C9
:1015B000A70A0F931F9300910B0210910C02209128
:1015C0000D0230910E0260277127822793271F9109
:1015D0000F910C94A70A0C94A20A0E94EB0A609344
:1015E0000702709308028093090290930A020C94F8
:1015F000430A60E070E0CB010C94ED0A0F931F9357
:1016000041E050E060E070E08A019B0104C0000FFF
:10161000111F221F331F8A95D2F7C901B8011F91EC
:101620000F910C94ED0A0F931F9341E050E060E09E
:1016300070E004C0440F551F661F771F8A95D2F7CC
:101640008091070290910802A0910902B0910A02CC
:101650008A019B01082B192B2A2B3B2BC901B801AE
:101660001F910F910C94ED0A0F931F9341E050E0EE
:1016700060E070E004C0440F551F661F771F8A9515
:10168000D2F74095509560957095809107029091A2
:101690000802A0910902B0910A028A019B01082365
:1016A00019232A233B23C901B8011F910F910C94E0
:1016B000ED0A0F931F9341E050E060E070E004C03A
:1016C000440F551F661F771F8A95D2F78091070236
:1016D00090910802A0910902B0910A028A019B012F
:1016E000082719272A273B27C901B8011F910F9105
:1016F0000C94ED0A0F931F930091070210910802BA
:101700002091090230910A02602B712B822B932BBE
:101710001F910F910C94ED0A0F931F9300910702F4
:10172000109108022091090230910A02602371236E
:10173000822393231F910F910C94ED0A0F931F9313
:1017400000910702109108022091090230910A02CB
:1017500060277127822793271F910F910C94ED0A20
:10176000089521E1929F800D1124E82FE695E695DA
:10177000E695877051E001C0550F8A95EAF785E03C
:10178000E89FF0011124EA53FE4F20E030E070E0C2
:101790004081CB01022E02C0969587950A94E2F70C
:1017A0008170819584278523842781932F5F3F4F04
:1017B0002530310569F7089521E1929F800D1124AC
:1017C000682F669566956695982F977085E0689F57
:1017D000B001112440E050E080E0FB01E40FF51F70
:1017E000EA53FE4F208130E0092E02C0369527953E
:1017F0000A94E2F721703327042E01C0220F0A94C5
:10180000EAF7822B4F5F5F4F4530510531F708955E
:10181000BF92CF92DF92EF92FF920F931F93CF93DD
:10182000DF938C01C0900702D0900802E09009027B
:10183000F0900A0280910B0290910C02A0910D028F
:10184000B0910E02C82AD92AEA2AFB2ACFE1D0E0B9
:10185000D701C6010C2E04C0B695A795979587951C
:101860000A94D2F780FD04C0219790F7B12C07C0ED
:10187000BC2EB8018C2F0E947D130197A9F38B2DEC
:10188000DF91CF911F910F91FF90EF90DF90CF905C
:10189000BF900895CF93DF93EC010E94080CBE0126
:1018A0000E947D13DF91CF9108951F93CF93DF9313
:1018B000EB019091C501992321F0CB010E944A0CC4
:1018C00013C0882349F0CB010E94080C182F682F01
:1018D000CE010E94B10B04C0CB010E94DC0B182F7B
:1018E000BE01812F0E947D13DF91CF911F9108953A
:1018F0001F93CF93DF93C0910F0216E080911002E7
:10190000C81799F0D0E01C9FF0011D9FF00D112425
:10191000EF5EFD4F408151816281738184819581A9
:101920000E94910A2196C770E9CFDF91CF911F9154
:10193000089540914102509142026091430270919A
:10194000440280914502909146020C94910AEF92D4
:10195000FF920F931F93CF93DF938091460282955E
:101960008F7009F065C080914302882309F460C03C
:1019700080910F02F09010021091410200914202FA
:10198000609144027091450291E01F3F09F090E0A0
:10199000C0910001D0910101292F96E0E92E8F1509
:1019A00009F446C06115710521F00F3F21F030E0C8
:1019B00003C031E001C0322F90E030FD36C0E89E18
:1019C000F001E99EF00D1124DF01AF5EBD4F1196CD
:1019D0003C911197301329C03C91311326C01296C7
:1019E0003C911297311121C013964D915C9114973F
:1019F000461B570B4C175D07C0F4809146028F7051
:101A0000806180934602EA5EFD4F80818F70806125
:101A1000808381E492E00E940F0ADF91CF911F91B1
:101A20000F91FF90EF900C94780C01968770B7CFD0
:101A3000DF91CF911F910F91FF90EF9008959F92AA
:101A4000AF92BF92CF92DF92EF92FF920F931F93CC
:101A5000CF93DF93CDB7DEB761970FB6F894DEBFB3
:101A60000FBECDBF8C0185E0F801DE011D9601900F
:101A70000D928A95E1F7D8011296EC90909141026F
:101A8000E091420220914402309145022115310536
:101A900031F0EF3F31F481E09F3F19F403C081E062
:101AA00001C080E0B82FB1709B2E80FD47C1D801E6
:101AB0004C9111965C9111971396AD90BC90149730
:101AC00081E4C82E82E0D82EF0904302B501621B5B
:101AD000730B2091000130910101FF2009F4D9C05E
:101AE000809146026217730708F095C0282F207F67
:101AF00009F052C05E1313C0491311C0FE2CE1104F
:101B00000EC08F708061809346020E94990CC601BE
:101B10000E940F0A80914602F80185834DC1AB28CF
:101B200031F05F3F31F481E04F3F19F403C081E0B1
:101B300001C080E080FD03C081E08E2502C080E00E
:101B400090E0F82FF170FF2E80FF1CC080910F02F3
:101B50002091100236E0821709F40BC190E0389F03
:101B6000F001399FF00D1124EF5EFD4F6181561396
:101B700006C06081461303C06281E61203C001966D
:101B80008770E9CFFE2CEE2009F416C18091460241
:101B900081608093460254C05E1306C0491304C09E
:101BA000E11002C0F80199C0C8010E947A0A882396
:101BB00061F1EE2051F120914602822F82958F70C3
:101BC00090E0029774F080914102909142029887D0
:101BD0008F831986BB86AA862C87CE0107960E9422
:101BE0000F0A86E0F801A1E4B2E001900D928A9517
:101BF000E1F70E94A70C0E94990C0AC05E1711F130
:101C0000C8010E947A0A81112CC0C8010E940F0AE3
:101C1000FF24F394D1C0282F207F81F77A2DB98A31
:101C2000A88A6E2D89890E94820A81E492E00E942E
:101C30000F0A86E0D6011D928A95E9F70E94990C59
:101C4000F12CBAC04913DCCFE110DACFF80185835B
:101C5000C8010E940F0A86E0D6011D928A95E9F715
:101C6000ABC0EE2091F220914602822F82958F70B8
:101C700090E002970CF4B5CF80914102909142021E
:101C80009A8389831B82BD82AC822E83CE0101960A
:101C9000A6CF6217730708F044C0FE2CEE2009F4AB
:101CA000B4CF5E1330C049132EC02091460220FDF0
:101CB00021C0822F82958F70482F50E04115510529
:101CC000C9F0F80125834F30510541F08F5F982FFF
:101CD0009295907F822F8F70892B8583C8010E94F7
:101CE0000F0A86E0F801A1E4B2E001900D928A9516
:101CF000E1F73CC086E0F801A1E4B2E001900D926A
:101D00008A95E1F759C0C8010E947A0A811169CF0A
:101D100080914602816080934602C8010E940F0AAA
:101D20004BC07A2DB98AA88A6E2D89890E94820AB1
:101D300086E0D6011D928A95E9F718C0EE2009F4D5
:101D400064CFC8010E947A0AF82E882309F45DCF77
:101D500086E0F801A1E4B2E001900D928A95E1F7E6
:101D600081E492E00E947B060E94A70C0E94990CDD
:101D700023C04D875E878D859E850E944A0C292F42
:101D800022952F70223028F49F7039F0811105C000
:101D90000BC0243028F49F7049F4805E883020F016
:101DA000C8010E940F0A9F2CF92C06C0D801159675
:101DB0009C91907F91F7F8CF8F2D61960FB6F89494
:101DC000DEBF0FBECDBFDF91CF911F910F91FF906E
:101DD000EF90DF90CF90BF90AF909F9008951F93AA
:101DE000CF93DF93CDB7DEB72C970FB6F894DEBF55
:101DF0000FBECDBF4F83588769877A878B879C87B3
:101E0000CE0107960E941F0D8823D1F09F818885FF
:101E10002A853B85232B31F08F3F31F481E09F3FB2
:101E200019F403C081E001C080E080FD47C04F810C
:101E3000588569857A858B859C850E94910A3EC06C
:101E400086E0FE013796DE01119601900D928A958B
:101E5000E1F7FF81E8856A857B856115710531F0C1
:101E6000EF3F31F481E0FF3F19F403C081E001C08E
:101E700080E080FD23C02091100230E0C90101966E
:101E80008770992740910F0250E084179507F1F170
:101E9000F983EA837D836C8396E0929FD001939FC0
:101EA000B00D1124AF5EBD4FFE01319601900D9231
:101EB0009A95E1F7809310020E94780C16E08091C9
:101EC0000F0290911002891771F1189FC00111241F
:101ED0008F5E9D4F0E941F0D882329F1E0910F0214
:101EE0001E9FF0011124EF5EFD4F40815181628100
:101EF0007381848195810E94910A80910F0290E004
:101F000001968770992780930F02D9CF0E945B0AB0
:101F10001092100210920F02E1E4F2E086E0DF017D
:101F20001D928A95E9F72C960FB6F894DEBF0FBE86
:101F3000CDBFDF91CF911F91089580916702859564
:101F40008595859508958091670287700895909191
:101F50006702977081E009F480E0089580918A0219
:101F6000089590918A02892B80938A020895809522
:101F700090918A02892380938A02089510928A029E
:101F8000089590918902892B809389020895809504
:101F90009091890289238093890208951092890281
:101FA000089580916802089508950C94D40F0C94BC
:101FB000D50F9091F20292FD08C090916802981797
:101FC00021F0809368020C94D70F089580916802E5
:101FD000882329F01092680280E00C94D70F0895AE
:101FE000CF93DF93E0910201F091030180918A0287
:101FF0008083E0910201F091030190818091890238
:10200000892B808380916802882381F0E09102010E
:10201000F09103019081892B80838091020190913E
:1020200003010E948B1C81110E94E60FC0910201E6
:10203000D091030140E250E067E472E0CE010E94DB
:102040006325892B69F080E2FE01A7E4B2E00190EC
:102050000D928A95E1F7CE01DF91CF910C94371C58
:10206000DF91CF9108950C94D40F9091F20292FDDC
:1020700010C098E0899F90011124262B20936702BD
:102080000E94130B809167028595859585950C9428
:1020900033100C94130B1092670280E00C943310F1
:1020A000209167028095822380936702982F977012
:1020B00099F430E0482F082E000C550B24173507F3
:1020C00059F09091F20292FD07C08595859585950E
:1020D0000E94340B0C944B1008959091F20292FBE5
:1020E000222720F9281769F080FB92F99093F202D9
:1020F0008091F1029091F2020E94BB1082E00C9458
:10210000501008958091F20282FB882780F991E0B7
:1021100089270C946D1081E00C946D1080E00C9474
:102120006D106FEF7FEF80E090E00C949C2580E0D5
:1021300090E00E94782521E0893E9E4F09F020E042
:10214000822F089582E090E00C94702583E090E067
:102150000C947025CF9384E090E00E947025C82FE6
:1021600082E290E00E9470252C2F30E0A901582BCC
:10217000CA01CF910895CF93C92F682F84E090E0D2
:102180000E947E256C2F82E290E0CF910C947E25F8
:10219000AB01BC018FE090E00C949025AB01BC0139
:1021A00083E190E00C94902560E070E0CB010C940A
:1021B000CE1060E070E0CB010E94C8100C94D410E7
:1021C00069EE7EEF80E090E00E949C2560E082E076
:1021D00090E00E947E2560E083E090E00E947E25F2
:1021E00010920B0210920C0210920D0210920E022D
:1021F00060E084E090E00E947E2560E082E290E072
:102200000E947E2560E085E090E00E947E2560E0EF
:1022100086E090E00E947E256FEF87E090E00E94CC
:102220007E2540E050E0BA0188E090E00E949025D1
:1022300060E08DE090E00E947E2540E050E0BA0131
:1022400088E190E00E94902560E087E190E00E94A4
:102250007E2540E050E0BA018CE190E00E9490259C
:1022600060E070E080E290E00E949C2540E050E059
:10227000BA0188E190E00E9490250C94D9100C944A
:10228000E010682F8EE090E00C947E250E94F31DF4
:102290006093A7027093A8028093A9029093AA0268
:1022A0006093A3027093A4028093A5029093A60268
:1022B000089585B7806885BF85B7806885BF089514
:1022C00081E008950C94601108950C9464110C94AD
:1022D00064110C9467110C9464110C946B110C94A0
:1022E00064110E94591189E594E10E94211C0E9409
:1022F0006F110C946D110E9465110C9464110E9471
:1023000073140E9411060C9415040E94DE1D0E9495
:1023100007030E947F110E9487170C9469112F9266
:102320003F924F925F926F927F928F929F92AF9265
:10233000BF92CF92DF92EF92FF920F931F93CF93B2
:10234000DF93CDB7DEB72D970FB6F894DEBF0FBE83
:10235000CDBF0E943D03282E81110E9446118BE8BB
:1023600092E09D878C8700E010E0302E802F0E9445
:10237000FA022B013C01EC85FD8581919191A1919F
:10238000B191FD87EC875301420188269926AA2640
:10239000BB2681149104A104B104B1F40F5F1F4F57
:1023A0000630110511F78FEF89838A831B820E9403
:1023B000E71D8160782F9D838C8349815A816B81D1
:1023C0008D810E94310651C08091AB0281FD0E9437
:1023D00006031B86C12CD12C7601C394D501C40100
:1023E0008C219D21AE21BF21892B8A2B8B2B91F132
:1023F0000E9462118823D1F0FB85FE833F824C202E
:102400005D206E207F2081E045284628472809F47A
:1024100080E088870E94E71D8160782F9A878987EE
:102420004E815F8168858A850E943106000F111FE9
:10243000000F111FF801E557FD4F80819181A281A6
:10244000B381C826D926EA26FB26C082D182E28241
:10245000F3820BC08B858F5F8B87CC0CDD1CEE1C51
:10246000FF1C813109F0BACF99CF81E0211001C062
:1024700080E02D960FB6F894DEBF0FBECDBFDF9182
:10248000CF911F910F91FF90EF90DF90CF90BF9071
:10249000AF909F908F907F906F905F904F903F9004
:1024A0002F9008950E948F110E9455160C942606B5
:1024B000CF93DF930E948213EC01811521E59207EF
:1024C00008F045C0811530E5930708F094C0883EB8
:1024D000910528F5803E910508F0F8C0883A9105ED
:1024E00070F4853A910508F07CC08130910509F4BB
:1024F00075C008F4E8C0049708F0E8C0E4C08F3B5A
:10250000910508F0E0C0C85AD0E0CC0FDD1FCF59CC
:10251000DE4F0990D881C02DCE019464D8C08115BA
:1025200040E2940758F4811551E0950708F0CEC0B9
:102530008D3E910508F4C7C09065C9C0C11580E4FF
:10254000D80708F4C0C0DF70CE01906AC0C0811502
:1025500025E59207A8F4811534E5930708F095C0A6
:10256000811543E5940708F07BC0811552E5950776
:1025700008F061C0D82FCC27CE01816F906AA7C028
:10258000C11589E5D807A0F4C11528E5D20708F0E0
:1025900082C0C11536E5D30708F095C08C2F0E9484
:1025A00016148F7190E0D82FCC27CE0190628FC087
:1025B000C1154AE5D40708F474C0CE0190568115C0
:1025C000904208F080C08D2F8F710E941614DD2775
:1025D000D0628F71AE01582BCA0179C081E090E0C2
:1025E00076C0C55AD0E0C157DE4F8881C82FD0E0F1
:1025F000CE0190646CC074E0969587957A95E1F76A
:10260000282F23703C2F337081E090E002C0880FA8
:10261000991F3A95E2F79C68AC01522B9A019C2FC6
:102620009F709695969550E2959FE0011124C901FF
:102630008C2B9D2B4CC08370992721E030E002C089
:10264000220F331F8A95E2F79C2F9695969580E28C
:10265000989FE0011124C22BD32BCE019C6837C078
:102660008370992721E030E002C0220F331F8A9542
:10267000E2F79C2F9695969540E2949FE0011124F5
:10268000C22BD32BCE019A6822C0D82FCC27CE01E3
:10269000846F906A1CC0DC2FCC27CE01806F906ABB
:1026A00016C08C2F8F700E94161494E0D695C79593
:1026B0009A95E1F7CF70D0E0DC2FCC27D0699E014E
:1026C000282BC90104C080E090E001C0CE01DF9159
:1026D000CF91089526E6829FC0011124FC0121E1DB
:1026E000729FE00DF11D1124E60FF11DEE0FFF1F8B
:1026F000E458FE4F8591949108950E946A130E94B8
:10270000581208958238910569F1B0F4813391052A
:1027100009F46DC048F48932910509F463C08A3226
:10272000910509F469C008958533910509F455C0F0
:1027300089339105B9F00895833E910569F138F424
:10274000803E9105B1F0823E910509F10895863EE3
:102750009105A9F1873E9105B9F1843E910509F0F3
:1027600064C023C02091F10220FD4FC021FD4DC067
:1027700008958091F10280FD44C08091F20280FFB3
:1027800044C08091F10284FD42C083EE4DC080912F
:10279000F10282FF38C0F5CF8091F10282FD33C093
:1027A0008091F20280FD31C0ECCF8091F20281FF76
:1027B00032C08091F10284FD2AC087EE35C080913D
:1027C000F10283FF26C0F5CF8091F10283FD21C085
:1027D0008091F20281FD1FC0ECCF8091F10285FD56
:1027E0001CC01DC08091F10285FD19C016C08091EA
:1027F000F10286FD16C017C08091F10286FD13C05C
:1028000010C089E311C082EE0FC080EE0DC080E0E1
:102810000BC086EE09C084EE07C089E205C085E3DF
:1028200003C08AE201C081E390E008959091F10233
:1028300092FF0DC0282F2871283019F4877F8460FB
:1028400006C0282F2471243011F48B7F886093FFF9
:102850000DC0282F2871283119F4877E846106C0A5
:10286000282F2471243111F48B7E88612091F2028B
:1028700020FF0DC0382F3871383019F4877F816000
:1028800006C0382F3171313011F48E7F886021FFFE
:102890000DC0282F2871283119F4877E816106C068
:1028A000282F2171213111F48E7E886194FD877E5D
:1028B000089580E008950C9491100E943D038FE1EB
:1028C0009EE40197F1F700C000000E943D0380E004
:1028D0000E94FA0260FF04C00E945B140C94341E34
:1028E00008950C945D140E949710811102C00E94FB
:1028F0003F110E94A2108093AB020E94AA109093F5
:10290000F2028093F1020E9471140E94A610682FB7
:1029100070E080E090E00E94B30A6091070270913D
:1029200008028091090290910A020C94EB0A089522
:10293000FF920F931F93CF93DF93F82ED92F8B0124
:10294000C42F222349F081E08093AE020E94E71D4C
:102950009093AD028093AC028091AE028823F1F097
:102960008091AC029091AD020E94FF1D0597B0F0DE
:10297000EF2DFD2FD80180E090E04C2F50E0841720
:10298000950754F401911191219131910D931D936B
:102990002D933D930196F3CF1092AE02DF91CF912C
:1029A0001F910F91FF9008950E94FF1F0E948511B3
:1029B0000C940B200E940F200E9452120C9429208C
:1029C0000E94851D0E94E61F0E9471110E94D4146E
:1029D0000E94DA140E947B11FBCF8091B50280FF28
:1029E00006C06091090170E0660F771F26C081FF65
:1029F00004C06091090184E005C082FF07C06091B6
:102A0000090188E0689FB001112417C09091B402B9
:102A10009923D1F060910801961788F72091090158
:102A200088E0289F90011124929FA001939F500D50
:102A3000112470E0CA010E9435256038710540F408
:102A40006115710519F406C068E070E0862F0895DD
:102A50008FE7089581E008958091B50280FF08C056
:102A60006091050170E0759567957595679521C032
:102A700081FF06C06091050170E07595679519C0EA
:102A800082FF04C06091050170E010C09091B30214
:102A9000992399F0609104019617A0F780910501A0
:102AA000899FC001112470E00E94352560387105AE
:102AB00040F46115710519F406C061E070E0862FDD
:102AC00008958FE7089581E008958D3E21F40E94D6
:102AD000ED14819504C08E3E29F40E94ED1480937C
:102AE000B90208958F3E21F40E94ED14819504C02F
:102AF000803F29F40E94ED148093B8020895893F25
:102B000019F40E942C1505C08A3F31F40E942C153F
:102B100081958093BA0208958B3F21F40E942C1571
:102B2000819504C08C3F29F40E942C158093BB0230
:102B300008959FE0980F983078F421E030E0A901E3
:102B400002C0440F551F9A95E2F7CA019091B7024F
:102B5000892B8093B70208958D3F21F48091B502AF
:102B600081600BC08E3F21F48091B502826005C068
:102B70008F3F29F48091B50284608093B502089557
:102B80008D3E39F49091B90297FF35C01092B90289
:102B900059C08E3E29F49091B9021916BCF32BC08E
:102BA0009091B8028F3E29F497FF25C01092B80289
:102BB00049C0803F19F41916CCF31DC09091BA0298
:102BC000893F29F41916BCF41092BA023BC08A3F1F
:102BD00019F497FF10C0F8CF8B3F39F49091BB02E6
:102BE00097FF09C01092BB022DC08C3F21F4909139
:102BF000BB021916BCF39FE0980F983080F421E0D7
:102C000030E0A90102C0440F551F9A95E2F7CA01AE
:102C100080959091B70289238093B70213C08D3FAE
:102C200021F48091B5028E7F0BC08E3F21F48091FC
:102C3000B5028D7F05C08F3F29F48091B5028B7F4F
:102C40008093B5028091B802811106C08091B902CB
:102C5000811102C01092B4028091BA02811106C0A3
:102C60008091BB02811102C01092B30208950E94AC
:102C7000E71D2091B802211104C02091B90222233E
:102C800021F09093B2028093B1022091BA022111F7
:102C900004C02091BB02222321F09093B0028093C4
:102CA000AF0286EB92E00C94511CEF92FF920F93CF
:102CB0001F93CF93DF9300D000D000D0CDB7DEB705
:102CC00086E0E6EBF2E0DE01119601900D928A9526
:102CD000E1F7E090B802F090B9020091BA021091C9
:102CE000BB021092B8021092B9021092BA0210926E
:102CF000BB02E11003C0FF2009F45DC08091B10266
:102D00009091B2020E94FF1DAC019091B4029923F0
:102D100039F020910A0130E02417350758F04BC0F4
:102D200020910B018AE0289F900111242417350778
:102D300018F041C09F3F19F09F5F9093B402EE20BE
:102D400061F00E94ED141E1414F09FEF01C091E099
:102D5000989F902D11249093B802FF2061F00E945B
:102D6000ED141F1414F09FEF01C091E0989F902D77
:102D700011249093B9023091B8023323E1F02091ED
:102D8000B9022223C1F045EB3403C0011124992379
:102D900019F09093B80203C081E08093B80235EB3C
:102DA0002303C0011124992319F09093B90203C0A1
:102DB00081E08093B902011103C0112309F45DC0C1
:102DC0008091AF029091B0020E94FF1DAC019091E2
:102DD000B302992339F02091060130E0241735071A
:102DE00058F04BC0209107018AE0289F90011124E0
:102DF0002417350718F041C09F3F19F09F5F90934B
:102E0000B302002361F00E942C15101614F09FEFFE
:102E100001C091E0989F902D11249093BA02112344
:102E200061F00E942C15111614F09FEF01C091E083
:102E3000989F902D11249093BB023091BA023323B6
:102E4000E1F02091BB022223C1F045EB3403C00125
:102E50001124992319F09093BA0203C081E0809362
:102E6000BA0235EB2303C0011124992319F0909382
:102E7000BB0203C081E08093BB028091B802811144
:102E80000BC08091B902811107C08091BA028111F3
:102E900003C08091BB0281110E943716EB82FC8235
:102EA0000D831E8386E0FE013196A6EBB2E0019011
:102EB0000D928A95E1F726960FB6F894DEBF0FBE05
:102EC000CDBFDF91CF911F910F91FF90EF900895AB
:102ED000E6EBF2E086E0DF011D928A95E9F71092B9
:102EE000B4021092B3021092B502089586E090E009
:102EF0000C947025682F86E090E00C947E258091DC
:102F0000F302847089618093F3020C947A170E9413
:102F10009710811104C00E943F110E947F170E94E8
:102F200076178093F302282F26952695269530E074
:102F30002430310524F0877088618093F3028091FA
:102F4000F30280FF04C086958695869501C080E0D7
:102F50000C941B042091F302822F8695869586950A
:102F6000482F50E04330510554F48F5F982F990F4C
:102F7000990F990F822F8770892B8093F30280918C
:102F8000F30281608093F3020E947A178091F3022A
:102F90008695869586950C941B048091F302982F54
:102FA000969596959695A1F0915E990F990F990F28
:102FB0008770892B8093F302887F91E009F490E079
:102FC0008091F30290FB80F98093F3020E947A17BC
:102FD0008091F3028695869586950C941B048091CA
:102FE000F30280FD13C081608093F302813019F4F5
:102FF00089E08093F3028091F3020E947A17809116
:10300000F3028695869586950C941B04089580910D
:10301000F30280FF08C08E7F8093F3020E947A172C
:1030200080E00C941B0408958091F30280FD0C94C1
:1030300007180C94EF179091F302892F86958695C7
:1030400086958F5F8F719770843038F4880F880F62
:10305000880F892B8093F30202C09093F302809132
:10306000F302887F91E009F490E08091F30290FBF5
:1030700080F98093F3020E947A178091F30286957B
:10308000869586950C941B04843008F083E090911B
:10309000F3029770282F220F220F220F922B90936A
:1030A000F302987F21E009F420E09091F30220FBE5
:1030B00090F99093F3020C941B040E9444188091A1
:1030C000F3020C947A179C01FB018281882349F159
:1030D0002E3BFCE53F07C9F040F42C3BECE53E07F6
:1030E00069F02D3B3C4561F00895203C9CE5390793
:1030F00091F070F0213C3C4589F0089583E001C0D7
:1031000080E00E945D1880E008950E94CD17FBCFFB
:103110000E94AA17F8CF0E941418F5CF0E941B181E
:10312000F2CF81E00895CF93DF93EC01FB01828120
:10313000882309F43CC1C430FDE5DF0760F4CB3FD0
:103140009CE5D90788F49E0122503C452431310585
:1031500008F02EC109C0C236EDE5DE0729F0C63AF7
:10316000FDE5DF0709F024C10E94AA109093F20246
:103170008093F102C1318CE5D80709F4C6C008F08C
:1031800042C0C930ECE5DE0709F49BC000F5C5304C
:103190008CE5D80709F485C078F4C330ECE5DE0788
:1031A00009F478C008F07AC0C230DC4509F0F5C0F7
:1031B0008091F1028160EFC0C7309CE5D90709F426
:1031C00078C008F07AC08091F1028061E4C0CD300F
:1031D000FCE5DF0709F487C058F4CB309CE5D9073C
:1031E00009F479C008F07BC08091F10288606FC05B
:1031F000CF30FCE5DF0709F480C008F082C0809181
:10320000F102877FC8C0CE3F9CE5D90709F471C0A1
:1032100000F5C531FCE5DF0709F485C068F4C3316A
:103220009CE5D90709F475C008F095C00E945B0AB7
:103230008091F1028F77AFC0CC3FFCE5DF07A9F1A9
:1032400008F054C0CB3FDC4509F0A7C08091F202E2
:1032500040C0C230EDE5DE0709F489C058F4C1155D
:103260008DE5D80709F45AC008F069C08091F202D0
:1032700082602FC0C236EDE5DE0709F47CC0C63A95
:10328000FDE5DF0709F481C0C330DD4509F085C0E5
:1032900080E06EC08091F10282607DC08091F10279
:1032A00016C08091F102886076C08091F20282603F
:1032B0004FC08091F10280626EC08091F102806403
:1032C0006AC00E945B0A8091F102806864C08460D9
:1032D00062C081603DC08091F1028E7F5CC08091B0
:1032E000F1028D7F58C08091F10216C08091F202E8
:1032F00018C08091F2028D7F2BC08091F1028F7EE9
:103300004AC08091F1028F7D46C08091F1028F7B8F
:1033100042C08091F102877F8B7F3DC08091F20295
:103320008D7F8E7F15C08091F10282FB222720F9CC
:1033300091E0922790FB82F990FB83F92CC0809159
:10334000F202982F909591708E7F892B90FB81F9D6
:103350008093F20222C00E945B0A8091F10287FBF7
:10336000222720F991E0922790FB87F914C081E091
:103370000E94411112C08091F10284FB222720F9A2
:1033800091E0922790FB84F906C08091F102982F7A
:10339000909590FB80F98093F1028091F1029091D9
:1033A000F2020E94BB100E945B0A80E001C081E033
:1033B000DF91CF910895893289F1F0F4843171F170
:1033C000B0F4873009F077C081E080930B0184E18D
:1033D00080930A018AE0809309018EE180930801BD
:1033E00088E08093050188E28093040164C092EE36
:1033F000980F9A30F0F05FC0803509F444C028F48B
:103400008F3409F058C08AE03FC0813529F08235F9
:1034100009F051C081E038C08FEF36C08091BE0204
:10342000882379F11092BE021092BD021092BC0264
:1034300042C08D518093BE02833099F038F48130C0
:1034400069F08230D9F48AE091E00DC0853099F0BE
:1034500078F0863099F484E091E005C08BE091E04B
:1034600002C089E091E09093BD028093BC0223C02A
:1034700088E091E0F8CF85E091E0F5CF1092BE02B0
:103480001AC080E0089586EFE091BC02F091BD0281
:10349000309789F02081082E000C990B820F911D26
:1034A0008F3F910519F014F08FEF04C097FF02C011
:1034B000108201C0808381E008950F931F9341E043
:1034C00050E060E070E08A019B0104C0000F111F12
:1034D000221F331F8A95D2F7C901B8010E94B30A8F
:1034E0001F910F910C945B0A482F50E0FA01359719
:1034F000EF33F10508F060C0EE59FF4F0C944925F9
:103500000E943F1155C08091AB02817F8E7F8093D6
:10351000AB0281E08093BF0208950E94AE0448C0D0
:103520008091AB02982F9095917090FB80F98093D9
:10353000AB0291113DC0897F877F10C08091AB02A3
:1035400081FB222720F991E0922790FB81F980935B
:10355000AB02992369F18091AB0281608093AB0249
:1035600027C08091AB0282FB222720F991E09227AD
:1035700090FB82F9ECCF8091AB0283FB222720F9EC
:1035800091E0922790FB83F9E2CF0E945B0A809141
:10359000F10287FB222720F991E0922790FB87F91F
:1035A0008093F10205C0895301C08D510E945D1ABC
:1035B00081E0089580E0FACF80E0089580E00895EA
:1035C0000C94DE1ACF93C82F8091BF02813069F02E
:1035D00038F08230C1F58C2F0E94DB1981E039C0B0
:1035E0000E94AE0F823289F504C00E94AE0F823273
:1035F00061F48C2F0E94E01A811104C08C2F0E946C
:10360000741A1FC081E090E01CC08C2F0E94DE1A4B
:10361000811116C0C43189F058F4CB3089F0C03123
:10362000B1F482E08093BF0288E30E94DB1908C0F6
:10363000C93219F0C83321F00AC01092BF0207C086
:1036400081E0817006C01092BF0280E002C080E07D
:10365000F8CFCF910895CF93DF9386319C4541F504
:10366000EB010E94AE0F982F8A81209102013091C8
:103670000301882379F09A7A81E009F480E080934D
:10368000C002911102C069E201C065E3C9010E9454
:10369000211D0AC08091C002811102C069E201C0EF
:1036A00065E3C9010E942C1D0E94F00F80E001C05B
:1036B00081E0DF91CF9108950F931F93CF93DF9314
:1036C000C42FD22FFC0182818823C9F04093C3020A
:1036D0000E94E71D9093C2028093C10280E28C0F8A
:1036E000883008F057C0C77081E001C0880FCA95C4
:1036F000EAF7DF91CF911F910F910C94B807809159
:10370000C302481330C08091C1029091C2020E944E
:10371000FF1D883C910538F510E21D0FCD17B9F05B
:1037200080E28C0F883040F4C77081E001C0880FC0
:10373000CA95EAF70E94BF07183028F581E09D2F4F
:10374000977001C0880F9A95EAF70E94B807802FFA
:103750000E94AF071830F0F4D77081E001C0880FE5
:10376000DA95EAF70AC080E28C0F883098F4C770C7
:1037700081E001C0880FCA95EAF7DF91CF911F91D0
:103780000F910C94BF07802FDF91CF911F910F9164
:103790000C94AF07DF91CF911F910F9108950F9374
:1037A0009C01CB01243F4CE5340731F188F4293DDD
:1037B000FCE53F07D9F02A3D4CE5340779F1283D77
:1037C0003C45A9F506E221EE41EE68ED7CE52BC013
:1037D000263FFCE53F07E1F0A8F0273F3C4539F5DF
:1037E00007E225EE46EE67EF7CE51DC007E225EE19
:1037F00045EE69ED7CE517C006E221EE40EE64EF90
:103800007CE511C007E225EE44EE65EF7CE50BC0D8
:1038100006E221EE42EE66EF7CE505C008E221E01B
:1038200045EE6AED7CE50E945C1B80E008C0FC016F
:103830008281882319F01092C30201C081E00F91A8
:103840000895909393018093920108959093C902F3
:103850008093C8020895E091C802F091C9023097A0
:1038600021F00190F081E02D099480E00895E0912D
:10387000C802F091C902309799F0209118012223D3
:1038800059F02091F10227FF07C0DC012C9111961D
:103890002C93119726E02C930280F381E02D09945C
:1038A0000895E091C802F091C902309739F022E002
:1038B000DC012C930480F581E02D0994089520917A
:1038C000C6023091C7022817390771F09093C702DA
:1038D0008093C602E091C802F091C902309721F0AE
:1038E0000680F781E02D099408952091C40230915B
:1038F000C5022817390771F09093C5028093C4025E
:10390000E091C802F091C902309721F00084F1855E
:10391000E02D09940895FC013296809118018823C6
:1039200031F08091F10287FF02C09EE101C096E074
:1039300080E0915028F021912223D9F38F5FF9CFB5
:103940000895662351F1209118012223E9F0209176
:10395000F10227FF19C0462F4695469546954E31F0
:10396000E0F4677021E030E002C0220F331F6A9557
:10397000E2F7FC01E40FF11D828190E02823392356
:1039800081E0232B69F409C0FC013296089621914D
:10399000621729F0E817F907D1F780E0089581E070
:1039A00008959C01FC0132969FEF80E041914617FB
:1039B00089F09F3F19F4411101C0982F8F5F863025
:1039C000A9F79F3F39F0F901E90FF11D97FDFA952D
:1039D0006283089508959C012A5F3F4FFC01428154
:1039E000461301C01282019682179307B9F7089512
:1039F000262F2695269526952E3168F4FC01E20F98
:103A0000F11D677021E030E001C0220F6A95EAF7EE
:103A10008281282B22830895262F26952695269588
:103A20002E3170F4FC01E20FF11D677021E030E0EF
:103A300001C0220F6A95EAF720958281282322830C
:103A4000089520911801222329F02091F10227FDE9
:103A50000C94F81C0C94D11C20911801222329F0FD
:103A60002091F10227FD0C940C1D0C94EB1C20916D
:103A70001801FC013296222331F08091F10287FF78
:103A800002C08EE101C086E0DF011D928A95E9F750
:103A9000089508950C94491D83E08093CA020C9404
:103AA0004A1D811102C081E001C082E08093CA02F8
:103AB0000C944A1D0C94511D81E08093CA020C9411
:103AC0004A1D0C945C1D08950C94631D0C94641D98
:103AD0000C94631D0C94631D0C94631DCF930E9482
:103AE0006A1D0E943D030E94681DC0E08C2F0E9449
:103AF000FA02672B682B692B29F4CF5FC630B1F728
:103B000080E001C081E0CF91089508951F920F9247
:103B10000FB60F9211248F939F93AF93BF93809111
:103B2000CB02811113C08091F4029091F502A09113
:103B3000F602B091F7024196A11DB11D8093F402E7
:103B40009093F502A093F602B093F702BF91AF9164
:103B50009F918F910F900FBE0F901F90189580919D
:103B6000FC02843031F10E9416051092CB0220E451
:103B700088E190E00FB6F894A895809360000FBE9E
:103B80002093600083B7817F846083BF83B78160A7
:103B900083BF7894889583B78E7F83BF0FB6F894E0
:103BA000A895809160008861809360001092600009
:103BB0000FBE08950E945B0A0C941D0582E084BD2F
:103BC00093E095BD9DE797BD80936E0008952FB754
:103BD000F8948091F4029091F502A091F602B091D0
:103BE000F7022FBF08952FB7F8946091F4027091F7
:103BF000F5028091F6029091F7022FBF08959C0183
:103C00004FB7F8948091F4029091F502A091F602DA
:103C1000B091F7024FBF821B930B089578941F92C7
:103C20000F920FB60F9211248F939F93AF93BF9370
:103C30008091F4029091F502A091F602B091F70202
:103C40000196A11DB11D8093F4029093F502A093FB
:103C5000F602B093F702BF91AF919F918F910F90B1
:103C60000FBE0F901F90189581E08093E00080E2D6
:103C70008093D8001092C9008FE097E20197F1F786
:103C800000C0000087E090EBDC0180930503909377
:103C90000603A0930703B09308039CE088E10FB6E6
:103CA000F894A895809360000FBE90936000FFCFBA
:103CB0008091EF020895089522E02093E9002FEF0C
:103CC0003091E800215035FD06C03AE63A95F1F70B
:103CD00000C02111F5CF2091E80025FF0BC040E086
:103CE00050E066E070E00E949A208091E8008E77B4
:103CF0008093E8000895CF93DF9320911801222349
:103D000039F02091F10227FF03C060E222E002C0F7
:103D100068E021E02093E9002FEF3091E800215086
:103D200035FD06C03AE63A95F1F700C02111F5CF0E
:103D30002091E80025FF1DC0EC0180911801811140
:103D400005C040E050E068E070E003C070E040E093
:103D500050E0CE010E949A208091E8008E778093F7
:103D6000E80080E2FE01AFECB2E001900D928A958E
:103D7000E1F7DF91CF9108958093CC027093CE024A
:103D80006093CD028091FC02843001F582E0809343
:103D9000E9008FEF9091E800815095FD06C09AE60A
:103DA0009A95F1F700C08111F5CF8091E80085FF69
:103DB0000DC040E050E063E070E08CEC92E00E94C7
:103DC0009A208091E8008E778093E8000895BC01E6
:103DD00084E00C94BC1EBC0183E00C94BC1E80915A
:103DE000FB02811109C00E942B220E94882280912F
:103DF000E20084608093E20008951092FB0208952F
:103E00000C94611D6091F80281E0611101C080E0B5
:103E10000C944C1D9091FC0281E0943009F080E0FC
:103E20006091F8020C94511D42E061EC81E00E9427
:103E3000A42142E261EC82E00E94A4219091FC0264
:103E400081E0943009F080E06091F8020C945A1DF2
:103E50008091FE02833009F461C030F4813071F04A
:103E6000823009F49AC008958A3009F486C08B30F4
:103E700009F46CC0893009F0A8C020C08091FD020F
:103E8000813A09F0A2C08091E800877F8093E80022
:103E90008091010390910203892B21F460E28FEC61
:103EA00092E003C060E080E090E070E00E94E520D6
:103EB0008091E8008B778093E80008958091FD025F
:103EC000813209F082C08091010390910203029730
:103ED00008F07BC08091E800877F8093E8008091A4
:103EE000E80082FD05C08091FC028111F8CF6DC011
:103EF0002091F3008091F20090E0922B029731F430
:103F00008091F100813011F0863021F48091F10030
:103F10008093EF028091E8008B7753C08091FD027F
:103F2000813A09F052C08091010390910203892BDC
:103F300009F04BC08091E800877F8093E800809172
:103F4000E80080FFFCCF8091180136C08091FD020F
:103F50008132D9F58091010390910203892BA9F553
:103F60008091E800877F8093E8000E94D9218091AA
:103F7000FF02809318010C945B0A8091FD0281324C
:103F800021F58091E800877F8093E8000E94D92185
:103F9000809100038093F00208958091FD02813AA0
:103FA000A1F48091E800877F8093E8008091E80089
:103FB00080FFFCCF8091F0028093F1008091E800B7
:103FC0008E778093E8000C94D921089584B7877F79
:103FD00084BF0FB6F894A8958091600088618093A3
:103FE0006000109260000FBE90E080E80FB6F89479
:103FF00080936100909361000FBE0C945C1D0E9441
:104000002B220E948822E2EEF0E08081846080838F
:1040100078940C941A258CE091E00C94261C8091E5
:10402000FC028530A9F48091FC02853079F40E946D
:10403000AF1D8091FA028823B1F30E946E1D882380
:1040400091F30E9485200E945B0AEDCF0C94DA1D4B
:10405000089508950C942C20292F332723303105FF
:10406000C9F060F42130310581F02230310509F0CA
:1040700044C08BE390E028EE33E043C021323105A9
:10408000E1F02232310549F138C082E190E023E2CB
:1040900034E037C099278130910549F028F0029724
:1040A00061F5E4ECF3E005C0E4EEF3E002C0E0ED1E
:1040B000F3E0849190E09F0124C06115710541F007
:1040C00061307105D1F489E090E023E134E019C05A
:1040D00089E090E02AEF33E014C06115710541F0EA
:1040E0006130710551F486EB90E025E334E009C0BE
:1040F00080E490E02BEE34E004C080E090E020E02B
:1041000030E0FA0131832083089519BC82E089BD33
:1041100009B400FEFDCF8091D8008F7D8093D80038
:104120008091E00082608093E0008091E00081FD5A
:10413000FCCF0895CF92DF92EF92FF920F931F93DF
:10414000CF93DF93EC018B017A010E94F82181115A
:1041500033C0E114F10439F0F70180819181081B2B
:10416000190BC80FD91FC12CD12C0115110519F13C
:104170008091E80085FD16C08091E8008E778093DD
:10418000E800E114F10449F0F70180819181C80E43
:10419000D91ED182C08285E00FC00E94F8218823F9
:1041A00021F30AC089918093F10001501109FFEFBA
:1041B000CF1ADF0ADACF80E0DF91CF911F910F9104
:1041C000FF90EF90DF90CF900895209103033091FE
:1041D00004032617370748F06115710539F420915B
:1041E000E8002E772093E80001C0B901FC0120E02F
:1041F0006115710579F18091FC028823F1F1853018
:10420000F1F18091E80083FD3CC08091E80082FDDF
:104210002EC08091E80080FFEBCF2091F3008091C9
:10422000F20090E0922B6115710551F088309105F4
:1042300038F421912093F100615071090196F3CF78
:1042400021E0089709F020E08091E8008E778093C4
:10425000E800CECF2111CFCF0AC08091FC02882385
:1042600061F0853061F08091E80083FD0AC08091A3
:10427000E80082FFF2CF80E0089582E0089583E0B5
:10428000089581E0089520910303309104032617D7
:10429000370748F06115710539F42091E8002E7751
:1042A0002093E80001C0B901FC0120E0611571050F
:1042B00091F18091FC02882309F440C0853009F413
:1042C0003FC08091E80083FD3DC08091E80082FD01
:1042D0002FC08091E80080FFE9CF2091F30080910A
:1042E000F20090E0922B6115710559F0883091052C
:1042F00040F424912093F1003196615071090196A8
:10430000F2CF21E0089709F020E08091E8008E7755
:104310008093E800CBCF2111CCCF0AC08091FC0262
:10432000882361F0853061F08091E80083FD0AC048
:104330008091E80082FFF2CF80E0089582E0089546
:1043400083E0089581E00895982F973068F5909361
:10435000E900981739F07091EC002091ED00509130
:10436000F00003C0242F762F50E021FD02C09F5F94
:10437000ECCF3091EB003E7F3093EB003091ED00BD
:104380003D7F3093ED003091EB0031603093EB00D6
:104390007093EC002093ED005093F0002091EE001C
:1043A00027FDE5CF80E008958F708093E90081E0DC
:1043B00008958091FD0287FF11C08091E80082FD81
:1043C00005C08091FC028111F8CF11C08091E800F6
:1043D0008B770BC08091FC02882349F08091E80024
:1043E00080FFF8CF8091E8008E778093E8000895F1
:1043F0002091E4003091E50095E64091EC00842F97
:10440000817040FF23C08091E80080FD1DC0809135
:10441000FC02882399F0853099F08091EB0085FDAE
:1044200011C04091E4005091E5002417350729F3AD
:10443000915011F09A01E1CF84E0089582E008954F
:1044400083E0089581E0089580E008954091E800B8
:1044500042FFDDCF08950E9499220E94A122E0EE42
:10446000F0E0808181608083E8EDF0E080818F77EB
:10447000808319BCA7EDB0E08C918E7F8C938081F6
:104480008F7E80831092FB0208950F931F93CF932A
:10449000DF930E9499220E94A122C8EDD0E088817A
:1044A0008F77888388818068888388818F7D8883DF
:1044B00019BC1092FC021092F8021092FA021092AB
:1044C000F90200EE10E0F80180818B7F8083888103
:1044D0008160888342E060E080E00E94A421E1EEF8
:1044E000F0E080818E7F8083E2EEF0E08081816069
:1044F0008083808188608083F80180818E7F8083C3
:10450000888180618883DF91CF911F910F910895F9
:10451000E8EDF0E080818F7E8083E7EDF0E0808140
:104520008160808384E082BF81E08093FB020C94F1
:104530004522E8EDF0E080818E7F80831092E200DA
:1045400008951092DA001092E10008951F920F92E0
:104550000FB60F9211242F933F934F935F936F9356
:104560007F938F939F93AF93BF93EF93FF9380912C
:10457000E10082FF0BC08091E20082FF07C08091C2
:10458000E1008B7F8093E1000E9419258091DA0081
:1045900080FF1DC08091D80080FF19C08091DA0093
:1045A0008E7F8093DA008091D90019BC80FF0BC008
:1045B00082E089BD09B400FEFDCF81E08093FC025A
:1045C0000E94EF1E04C01092FC020E94FD1E80910A
:1045D000E10080FF19C08091E20080FF15C080914A
:1045E000E2008E7F8093E2008091E2008061809300
:1045F000E2008091D80080628093D80019BC85E0E9
:104600008093FC020E94021F8091E10084FF2FC072
:104610008091E20084FF2BC019BC82E089BD09B4FF
:1046200000FEFDCF8091D8008F7D8093D8008091CF
:10463000E1008F7E8093E1008091E2008F7E809385
:10464000E2008091E20081608093E2008091F802B4
:10465000882311F084E007C08091E30087FD02C049
:1046600081E001C083E08093FC020E940A1F8091D8
:10467000E10083FF29C08091E20083FF25C0809183
:10468000E100877F8093E10082E08093FC0210923A
:10469000F8028091E1008E7F8093E1008091E2003A
:1046A0008E7F8093E2008091E20080618093E2003F
:1046B00042E060E080E00E94A4218091F0008860E8
:1046C0008093F0000E94001FFF91EF91BF91AF9186
:1046D0009F918F917F916F915F914F913F912F911A
:1046E0000F900FBE0F901F9018951F920F920FB64C
:1046F0000F9211242F933F934F935F936F937F9368
:104700008F939F93AF93BF93CF93DF93EF93FF93D9
:10471000C091E900CF708091EC00D82FD17080FD5E
:10472000D0E81092E9008091F000877F8093F0003C
:1047300078940E94B9231092E9008091F00088607B
:104740008093F000CD2BCF70C093E900FF91EF91E3
:10475000DF91CF91BF91AF919F918F917F916F9199
:104760005F914F913F912F910F900FBE0F901F902F
:1047700018951F93CF93DF93CDB7DEB7AA970FB6E7
:10478000F894DEBF0FBECDBFEDEFF2E08091F100F7
:10479000819323E0E530F207C9F70E94281F80913A
:1047A000E80083FF2EC18091FD029091FE02492F07
:1047B00050E04A30510508F024C1FA01EF55FF4F8F
:1047C0000C944925803821F0823809F01AC108C0BC
:1047D0008091F9029091FA02992389F082600FC0CA
:1047E000809101038F70873008F00BC18093E9003E
:1047F0008091EB0085FB882780F91092E900909169
:10480000E800977F9093E8008093F1001092F10008
:10481000D1C0282F2D7F09F0F4C0882319F08230F1
:1048200061F0EFC08091FF02813009F0EAC093305F
:1048300009F080E08093FA022EC08091FF0281117E
:104840002AC0809101038F702FEF280F263008F0C7
:10485000D8C08093E9002091EB0020FF1CC093306A
:1048600021F48091EB00806214C09091EB00906184
:104870009093EB0021E030E0A90102C0440F551FE6
:104880008A95E2F74093EA001092EA008091EB00EB
:1048900088608093EB001092E9008091E800877FA8
:1048A0008093E8000E94D921ACC08111AAC0109168
:1048B000FF021F778091E3008078812B8093E300D3
:1048C0008091E800877F8093E8000E94D921809141
:1048D000E80080FFFCCF8091E30080688093E300D4
:1048E000111102C082E001C083E08093FC0289C004
:1048F0008058823008F085C08091FF0290910003BB
:104900008C3D53E0950779F583E08A838AE28983B9
:104910004FB7F894DE01139620E03EE051E2E32F1A
:10492000F0E050935700E49120FF03C0E295EF7050
:104930003F5FEF708E2F90E0EA3010F0C79601C015
:10494000C0968D939D932F5F243149F74FBF80917F
:10495000E800877F8093E8006AE270E0CE0101966C
:104960000E94E52016C06091010370910203AE0120
:104970004F5F5F4F0E942A20BC01892B09F441C080
:104980009091E800977F9093E80089819A810E9436
:1049900043218091E8008B778093E80032C0803813
:1049A00081F58091E800877F8093E8008091F8028C
:1049B0008093F1008091E8008E7772CF811121C041
:1049C0008091FF029091000399270297D4F480917F
:1049D000E800877F8093E8008091FF028093F802CF
:1049E0000E94D9218091F802811106C08091E300D4
:1049F00087FD02C081E001C084E08093FC020E9438
:104A0000141F8091E80083FF0AC08091E800877F2F
:104A10008093E8008091EB0080628093EB00AA967F
:104A20000FB6F894DEBF0FBECDBFDF91CF911F91BF
:104A300008950895CF938091FC028823A1F0C0913E
:104A4000E900CF709091EC00892F817090FD80E893
:104A5000C82B1092E9008091E80083FD0E94B923E1
:104A6000CF70C093E900CF91089597FB072E16F4FD
:104A7000009407D077FD09D00E944F2507FC05D090
:104A80003EF4909581959F4F0895709561957F4F65
:104A90000895EE0FFF1F0590F491E02D0994AA1BD5
:104AA000BB1B51E107C0AA1FBB1FA617B70710F019
:104AB000A61BB70B881F991F5A95A9F7809590954B
:104AC000BC01CD010895FB01DC0104C08D91019072
:104AD000801921F441505040C8F7881B990B089564
:104AE000F999FECF92BD81BDF89A992780B50895B6
:104AF000A8E1B0E042E050E00C94A425262FF999FB
:104B0000FECF92BD81BDF89A019700B4021639F02C
:104B10001FBA20BD0FB6F894FA9AF99A0FBE0895FD
:104B20000396272F0E947F250E947E25252F0E9415
:104B30007F25242F0C947F250196272F0E947F2507
:104B40000C947E25DC01CB01FC01F999FECF06C057
:104B5000F2BDE1BDF89A319600B40D92415050403B
:084B6000B8F70895F894FFCFA7
:104B6800C8006902280850011E0A1401581E7B1E3D
:104B78005C1EEB1EE71E5B1E01366667F1F035FF13
:104B8800FFFFFFFFFFFFFFFFFFFF90919293953715
:104B9800E200E900EA00B500B600B700CD008301E5
:104BA800CC008A01920194012102230224022502E9
:104BB800260227022A02B300B4006F007000818227
:104BC80083E200E900EA00B500B600B700CD008333
:104BD80001CC008A019201940121022302240225BA
:104BE80002260227022A02B300B4006F0070008177
:024BF8008283B6
:00000001FF
